:03000000020030CB
:03000B00020119D6
:1000300011E020B0025132300021C200EA9002F3F8
:1000400093FBBB0A05115E02005BBB0B05118F021F
:10005000005B00A60308B878027870020037787059
:10006000760008B878FA787022E5301475F008A4A4
:10007000F53086F0E530517B510E080530B878F246
:10008000115EC201C20220B103D29622C29622782A
:10009000702001D57530017B00EB514B86F0B5F037
:1000A000300B08B878F3115EE530B40107D203D203
:1000B000023149227440514BB40005B2B1B29622CC
:1000C000C28CD2B1C29631F1115ED296C2B1D28C3D
:1000D000220B08B878FB78700530BB40BC115E225B
:1000E000D2B0D2B7D290D291D292C295C294C293DA
:1000F000D296C2007A00C2B1C202C203C2017534F4
:1001000001115E758901C288C2A8D28CD2A975324C
:10011000257533FF5124D2AF22758A71758CB2C018
:10012000E0C0F031A0D53411200306753406020179
:1001300034753401300202B296200208D53605111A
:100140005E753699D0F0D0E0323000FDC200EA9002
:1001500002F393FBBB0B0302018EBB000302018E73
:10016000BB0A0302018EBB0930C2033000FBC20090
:10017000EA9002F393FBB40A0302018EB40B03026C
:10018000018E75F002A4C5F07440517B510EC2027D
:1001900020B103D29622C29622D201C2038B302212
:1001A000D294D293C29531DE75F000701CD295C204
:1001B0009431DE75F0047011D294C29331DE75F083
:1001C00008D2937004E40201CB25F0B5020122CAE3
:1001D000700BD200753699C28C511ED28C227401DC
:1001E00030B70D043090090430910504309201E4D9
:1001F000227531FF7535FF7440514BD531FD753196
:10020000FFD535F77531FF7535FFD5E0EE22753135
:10021000FF753515D531FD7531FFD535F7227532AE
:1002200025753315B2B3D532FD753225D533F5D2E8
:10023000B322753700E537900300510E93F5F0E5D2
:1002400037517B0537E537B441F022C0F0F5F05166
:10025000D6402574A04400C2E0519F4019E5F051FA
:100260009F401351D6401174A04400D2E0519F40EA
:100270000551C1C3800251EAD0F02251D6401FC0BF
:10028000E074A04400C2E0519F400FD0E0C0E051B4
:100290009F4007E5F0519F4001C351EAD0E022C0E2
:1002A000F075F0083392B500D2B400C2B4D5F0F4C2
:1002B000D2B50000D2B400000000A2B5C2B4D0F0A4
:1002C00022D2B5C0F075F008D2B400A2B533C2B4E2
:1002D000D5F0F5D0F022D2B5D2B430B50B30B40899
:1002E000C2B500C2B4C38001D322C2B500D2B400EB
:1002F000D2B522FF0104070A020508000306090B14
:1003000001020304000000000202020200000000DB
:1003100003030303000000000404040400000000C1
:1003200005050505000000000606060600000000A1
:100330000707070700000000080808080000000081
:0103400002BA
:00000001FF
